:020000040000fa
:10800000f03f0020c9900000d39200004795000087
:108010000000000000000000000000000000000060
:108020000000000000000000000000004784000085
:10803000000000000000000047840000ed990000ef
:108040000000000000000000000000000000000030
:108050000000000000000000000000000000000020
:108060000000000000000000000000000000000010
:108070000000000000000000000000000000000000
:1080800000000000000000000000000000000000f0
:1080900000000000000000000000000000000000e0
:1080a00000000000000000000000000000000000d0
:1080b000000000000000000047840000478400002a
:1080c00047840000478400003d9700000000000046
:1080d00000000000000000000000000000000000a0
:1080e0000000000000000000000000000000000090
:0480f000000000008c
:020000040000fa
:1080f400f8b5c046f8bc08bc9e467047f99200002b
:10810400f8b5c046f8bc08bc9e467047d59200003e
:020000040000fa
:0881140008000000010000005a
:020000040000fa
:10811c00f0b51f0085b005000c0016000092019709
:10812c0002900391002f00d0d5e08e424ed9300042
:10813c0001f0c8f958b120232a001b1ada408440f8
:10814c001300864085402343009603930295009bc1
:10815c0003991a0cb1fbf2f615006b463700754308
:10816c001b884d1b5f4302992d040c0c25433100d9
:10817c00af4208d9009c01392d19ac4203d8af424b
:10818c0001d9b11e2d19ef1bb7fbf2f46243bf1ad4
:10819c006a46634312893f043a432600934208d946
:1081ac00009d013e5219954203d8934201d9a61e57
:1081bc0052190904d31a31430a9a1ab1c3401360f5
:1081cc00002353600800019905b0f0bd1eb90123ce
:1081dc00b3fbf6f30093009801f074f9c0bb009b5d
:1081ec00e41a01230193009b1a0cb4fbf2f1160064
:1081fc006b460d004e431b88a41b5d43029e24045a
:10820c00360c34430f00a54208d9009e013fa41937
:10821c00a64203d8a54201d98f1ea419641bb4fb36
:10822c00f2f67243a41a6a46734312892404144367
:10823c003100a34208d9009a0139a418a24203d8ec
:10824c00a34201d9b11ea4183f04e31a3943b3e782
:10825c00009b20228340009323002f00121ad3404e
:10826c008540d740009a0295110cb3fbf1f56a4694
:10827c002e0012888440944656430a006a432743d2
:10828c009b1a1b043a0c13432a009e4208d9009ceb
:10829c00013a1b199c4203d89e4201d9aa1e1b19f4
:1082ac009e1bb6fbf1f5644669436c43761a3604a3
:1082bc00bfb237432b00bc4208d90099013b7f1851
:1082cc00b94203d8bc4201d9ab1e7f1812041a4321
:1082dc003c1b019287e78f4209d90a9b002b00d1e6
:1082ec00a9e0186059600023019319006ae738006f
:1082fc0001f0e8f8c8b9a74202d30100ae4208d891
:10830c00ae1bb542ad410121e41b6d42631b0393cf
:10831c0002960a9b0193002b00d153e7029a1a6034
:10832c00039a5a60002301934ce720231b1a0093f5
:10833c003b003700009a8340d7401f432300d340b3
:10834c002a0000998440ca40224394463a0cb3fb5d
:10835c00f2f41100864085406143019626005b1ab9
:10836c0061460295bdb26e43090c1b040b43210000
:10837c009e4207d9db1901399f4203d89e4201d98d
:10838c00a11edb199e1bb6fbf2f462436346b61ac0
:10839c006a46654393819289360416432300b5429d
:1083ac0007d9f619013bb74203d8b54201d9a31e30
:1083bc00f619090419436b469c88019b721b944661
:1083cc001a0c23008eb20d0c6c437343554372434d
:1083dc001e0c1219b218944202d9802464022d1971
:1083ec00140c9bb212046519d218ac4503d30bd1f3
:1083fc00029b934208d2019bed1bd61ab2429241ca
:10840c005242ad1a320001390a9b0193002b00d164
:10841c00d8e6029b009c9a1a63465d1b029b934212
:10842c00bf417f42ed1b2b00c240a340c5401a4305
:0a843c000a9b24c376e70a9b56e76b
:020000040000fa
:02844600fee74f
:020000040000fa
:10844800582100201c0000000000000086210020a8
:1084580001000000000000000020002004000000cf
:1084680000000000042000200c00000000000000b4
:108478001020002008000000000000001820002044
:10848800010000000000000020210020380000004a
:108498000000000020200020a000000000000000d4
:1084a80084210020020000000100000001000000fb
:1084b800742100200400000001000000c0200020fa
:1084c800c020002060000000010000000000000043
:1084d8003099000050990000109900000000000039
:1084e8000000000000000000000000000000000084
:1084f8000000000000000000000000000000000074
:108508000000000000000000000000000000000063
:108518000000000000000000000000000000000053
:10852800000000000000000000000000782100208a
:1085380004000000000000007c210020040000006e
:10854800000000001c2000200400000000000000c3
:10855800802100200400000000000000000000004e
:10856800000000002222222222222222222222226b
:020000040000fa
:10857800f7b58a8905000c0013075ed44b68002bf9
:1085880004dc0b6c002b01dc0020febde76a002f29
:10859800fad000232e682b6041f200031a4092b3f0
:1085a800606da3895b0705d56368c01a636b0bb15f
:1085b800236cc01a0200216a00232800e76ab84722
:1085c800a189431c06d12b681d2b30d82b4ada40d1
:1085d800d3072cd50023636023692360cb0404d51b
:1085e800431c01d12b6803b96065616b2e600029bb
:1085f800cad023004433994202d0280000f0acfbd3
:1086080000206063c1e70123216a2800b847431ca2
:10861800c7d12b68002bc4d01d2b01d0162b01d13c
:108628002e60b1e74023a2891343a381ade740231d
:108638000b430120a3814042a7e70f69002fa3d075
:108648000b680f60db1b01930023920700d14b6975
:10865800a360019b002b00dc96e7019b3a00216a8e
:108668002800a66ab047002803dc4023a2891343e8
:10867800dfe7019b3f181b1a0193eae7010040203e
:020000040000fa
:10868800344b70b51d6806000c0025b1ab6913b9f1
:10869800280000f063fc304b9c420fd16c680c231f
:1086a800e25e93b219072cd4d90611d4092333609a
:1086b800402301201343a381404270bd274b9c42b5
:1086c80001d1ac68ebe7264b9c42e8d1ec68e6e7c1
:1086d8005b0712d5616b41b123004433994202d044
:1086e800300000f039fb002363632422a3899343fd
:1086f800a38100236360236923600823a2891343ad
:10870800a38123695bb940f2802140f20022a3894a
:108718000b40934203d02100300000f0e3fb01231b
:10872800a28913408bb10023a36063695b42a361f4
:1087380023690020002bc0d10c23e25e1306bcd5b0
:1087480040231343a3810138b7e7920700d4636934
:10875800a360ede7742100203099000050990000d3
:048768001099000064
:020000040000fa
:10876c00f0b5de4657464e464546e0b585b08446e4
:10877c00304b196b00285ad083689a4661b18b68cc
:10878c005246039240f200089a4548d30022002337
:10879c008b460092019306e052468260254b18638b
:1087ac00012035e0cb465e46b66834000025009ac1
:1087bc00019b12196b41009201935e46b669b1465a
:1087cc009eb14e46b66800210f00009a019bb61868
:1087dc005f41474503d8e5d1039b9e42e2d95946f8
:1087ec00009a019b48464c4602e059463000340042
:1087fc00b9b16446a0618c61002051468a1a634667
:10880c009a609b6923b1624691689a68521a9a6081
:10881c0005b03cbc90469946a246ab46f0bd0c0058
:10882c0000220448614601638c610120e5e70020c9
:08883c00eee7c04620210020f8
:020000040000fa
:10884400f8b5334c266b63689b699847606160692f
:1088540001f002f9050001f0f1f8002e4fd02c4c84
:108864002c22a35c0133a354280000f009ff246bdd
:108874002cb1a3681bb901250027254e11e0254e14
:108884000024370035001fe0e06900f03dfee36896
:108894000bb120699847346b002cf0d0a368002bef
:1088a400edd125756575a37813b9e368002bebd179
:1088b400200000f02ffca378002be8d16770e6e7d6
:1088c40001342036052c15d06301fb185b7d002b89
:1088d400f6d06301eb1800215975b378012befd161
:1088e40062010c4b9c466244736893603000fff74e
:1088f4003bffe5e706492c228b5c013b8b5401f0de
:1089040007f9040000f0dcf9200001f00af9f8bdd1
:0889140020210020202000209a
:020000040000fa
:10891c0070b505000e0018b183690bb900f01cfb93
:10892c00ab69ac6813b9280000f016fb294b9c42cc
:10893c0019d16c680c23e25e42f200031a4205d195
:10894c001343a381226e244b13402366a3891b0778
:10895c0001d52369fbb921002800fff78ffed0b1a8
:10896c000120404270bd1d4b9c4201d1ac68e1e737
:10897c001b4b9c42ded1ec68dce7013b0136a3606b
:10898c00002b04daa269934216db0a2914d023685f
:10899c005a1c226019703178a3680029edd1013b73
:1089ac00a360002b0fda22000a21280000f01af82d
:1089bc00431cd5d00a20d5e72200280000f012f87d
:1089cc00431ce8d1cce70a2023685a1c226018709b
:1089dc00c8e7c04630990000ffdfffff5099000048
:0489ec0010990000de
:020000040000fa
:1089f000f8b505000e00140018b183690bb900f03a
:108a0000b1fa274b9c4230d16c68a369a360a3895b
:108a10001b0734d5236993b30c23e25e42f20003b3
:108a2000f7b2f6b21a4234d023682269981a636901
:108a3000984204db2100280000f01cfb28bba3683f
:108a40000130013ba36023685a1c22601f706369d8
:108a5000984204d0a389db0719d50a2e17d121002b
:108a6000280000f007fb90b10fe00e4b9c4201d1b3
:108a7000ac68cae70c4b9c42c7d1ec68c5e7210043
:108a80002800fff701fe0028c6d0012676423000fc
:108a9000f8bd1343a381226e044b13402366c3e742
:108aa000309900005099000010990000ffdfffff8f
:020000040000fa
:108ab000032370b5cd1c9d43083506000c2d1cd238
:108ac0000c25a9421bd8300001f094f8254a1468ff
:108ad0002100c1b9244c23681bb9300000f048ffc5
:108ae00020602900300000f043ff431c2dd10c23ef
:108af0003000336001f07ff803e0002de1da0c2351
:108b00003360002070bd0b685b1b1bd40b2b03d99b
:108b10000b60cc18256003e08c420fd163681360b2
:108b2000300001f068f8200007220b30231d90432d
:108b3000c31a002be6d05a42e250e3e74b68636069
:108b40000c00ede70c004968c3e70323c41c9c43f9
:108b5000a042dfd0211a300000f00aff431cd9d117
:0c8b6000c5e7c046782100207c210020e1
:020000040000fa
:108b6c00f0b583b006000d0001921f0008ab1c7815
:108b7c0000f09afd20b901246442200003b0f0bd3e
:108b8c00214b1b785bb2022b04d00124644200f011
:108b9c0029fdf2e795b3b54233d31c4b1b786bb16f
:108bac001a4b203301221948a030197841b10132f7
:108bbc0020338342f9d301246442e8e70022134bab
:108bcc000121197000215970197559759c705d60df
:108bdc000199d9601f61ad1b9d600d4909880c047a
:108bec004ff6ff7002401443dc61013189b28142bf
:108bfc0002d0074a1180cae70121fae70124644236
:108c0c00c5e701246442c2e7202100202020002077
:048c1c00842100208f
:020000040000fa
:108c200070b50c0000293fd010b10120404270bd4a
:108c30001f4d01223423ea540b686b60db689847b0
:108c4000e8601c4bb3fbf0f3a02090fbf3f0023084
:108c500028620423e3562b7200232b610122524227
:108c6000aa61154aea616b62ab622b632c22ab549a
:108c70006b681b680021114898476b681b6913b12a
:108c80000b4a906998470a4ce06963685b699847aa
:108c900063685b689847a0220021094800f04cfff8
:108ca000022323702000c2e701204042bfe7c046f4
:108cb000202100200048e801ffffff7f45880000d9
:048cc0002020002050
:020000040000fa
:108cc40070b5244b1a6b59691961002a37d093681f
:108cd400002b2ddb94681f4b5b69e41800261d4da7
:108ce4006b689b69984700230200296933b9814264
:108cf40004d901204042002112184b4115490d6a44
:108d04000021280080185941b14202d81ed1a04246
:108d14001cd9aa180f4bda610e4bdb6913b9012277
:108d24000c4bda610b4bd8695b685b69984770bd83
:108d3400084b5c69084b9c4664440026cfe7054b0e
:108d44005c69054b9c4664440026c8e7014bdc6122
:0c8d5400e2e7c04620210020ffffff7f67
:020000040000fa
:108d600070b5050079b10c1f2368002b00dae418f8
:108d7000280000f03fff1c4a13682bb963601460a1
:108d8000280000f038ff70bda34209d9216860189f
:108d90008342f3d118685b6841182160eee7130045
:108da0005a680ab1a242fad919685818a0420bd1e0
:108db00020680918581819608242e1d11068526879
:108dc000411819605a60dbe7a04202d90c232b60de
:108dd000d6e721686018824203d1106852684118b2
:0c8de000216062605c60cbe7782100201d
:020000040000fa
:108dec001e4a1f4b70b50021934203d219700133f8
:108dfc009342fbd1002503261a4803684168b3b996
:108e0c0059b383680c30bbb100230022845c9c54a2
:108e1c0001328a42fad333000b405a1e934189081f
:108e2c0059188900401803684168002be8d0826803
:108e3c000c303ab90029e0d059181d7001338b421f
:108e4c00fbd1dae70029e0d133000b405a1e9341e5
:108e5c008908591889004018e5e770bd20200020ca
:088e6c000020002048840000f2
:020000040000fa
:108e7400f8b51c4b07001e68b36913b9300000f045
:108e84006ff84836b4687368013b03d5336833b16f
:108e94003668f7e70c22a55e6db16434f4e704216b
:108ea400380000f05ffc30600028f1d10c2304008e
:108eb4003b602000f8bd01235b42e38120000123d5
:108ec4002566a3812560a560656025616561a5614e
:108ed40008222900583000f02dfe6563a563a564bf
:088ee400e564e6e7e89b0000ed
:020000040000fa
:108eec00f7b502268b8905000c00334206d023000f
:108efc0047332360236101236361f7bd01ab6a46ed
:108f0c0000f02cf9009907002800fff7cbfd30b9d1
:108f1c000c22a35e9a05f0d41e43a681e7e70d4b05
:108f2c00ab628023a28920601343a381009b206144
:108f3c006361019b4bb10e23e15e280000f032fd12
:108f4c0018b10123a2891343a381a0893843a081be
:088f5c00d3e7c046499b000069
:020000040000fa
:108f6400836913b5040043bb8364c3640365134b73
:108f7400134a1b6882620193984201d101238361e1
:108f84002000fff775ff60602000fff771ffa0600d
:108f94002000fff76dff0022e0600421606800f00c
:108fa40051f901220921a06800f04cf90222122192
:108fb400e06800f047f90123a36113bde89b0000ba
:048fc400499b0000c5
:020000040000fa
:108fc80070b5040000f072fb0125d0b1200000f05c
:108fd800ddf90400d8b14378002583b983680bb95b
:108fe800436883602c230b4ad35c63b9200000f0ec
:108ff800edf900232375637501236370002500f0e4
:10900800f3fa280070bd2000fff7acfbf1e701255b
:08901800f5e7c046202100200d
:020000040000fa
:1090200070b582b005000e001c0003b9e8b122b98a
:1090300001246442200002b070bd0d4bd8680023ab
:10904000002100f025f940f2e832002300f0e2f9b7
:109050000100009433002a000020fff787fd040080
:10906000431ce7d0fff7b0ffe4e701246442e1e7e7
:04907000202100209b
:020000040000fa
:109074000b6970b505000c000bb9002070bd18b168
:1090840083690bb9fff76cff0b4b9c4209d16c68e9
:109094000c22a35e002bf0d021002800fff76afa0f
:1090a400ece7064b9c4201d1ac68f1e7044b9c42cf
:1090b400eed1ec68ece7c04630990000509900000e
:0490c40010990000ff
:020000040000fa
:1090c80010b50c4b03b198470b4b03b19847fff70a
:1090d80089fe0a4a7f210a4b8b439360094b9847c4
:1090e800094b03b19847094b03b1984700f060f862
:1090f800fee7c046000000000000000000ed00e0b0
:109108000080000001920000000000000000000044
:020000040000fa
:1091180010b50100114b1a6bdab1824202d100225c
:1091280004e01a009369b3b19942fad18b691bb173
:1091380088689c68001998602ab18b69936100203f
:1091480000238b6110bd054b1a6b92691a630120cd
:10915800f6e70020f6e70020f4e7c04620210020cb
:020000040000fa
:1091680070b50e001d000e23c95e90b014000029d2
:1091780007da00232b60b3891b0611d440f20043a1
:109188000fe001aa00f078fb0028f2db4ff20002a2
:10919800029b1340054a9b185a4253412b60ede746
:1091a80040230020236010b070bdc04600e0ffffe0
:020000040000fa
:1091b80070b5002000f092fa012340f2e832002155
:1091c8000948fff729ff094c094d260000f0e6fc85
:1091d8002378002bfad0280000f08efc0422054bdf
:1091e800da6100233370f1e7599b000086210020e3
:0891f800ac9a000000300040b9
:020000040000fa
:1092000070b500260c4d0d4c641ba410a64209d16c
:109210000026fef76fff0a4d0a4c641ba410a642fd
:1092200005d170bdb300eb5898470136eee7b300a7
:10923000eb5898470136f2e70081000000810000fa
:08924000008100000481000020
:020000040000fa
:10924800002310b5040003604360836081810366d6
:10925800c28103614361836119000822583000f01c
:1092680067fc054b24626362044ba362044be36210
:10927800044b236310bdc046ed97000081950000a4
:08928800959700007d9b00009a
:020000040000fa
:10929000f7b5050c019393b21f006b439c46140c69
:1092a00086b277436643654366443c0ca419a342e7
:1092b00002d980235b02ed18260cbfb2019b240467
:1092c000e41943432000514375195918491903b053
:0292d000f0bdef
:020000040000fa
:0292d200fee7b5
:020000040000fa
:1092d40010b5054c237833b9044b13b1044800e0ae
:1092e40000bf0123237010bd58210020000000009e
:1092f40000000000034b10b51bb10349034800e014
:1093040000bf10bd000000005c2100200000000030
:020000040000fa
:1093140001220d4b1a6019000b691a42fcd10a4b49
:1093240058221a6003221a7347f60052da61332274
:109334009a720021054a116020225a721a00136998
:10934400002bfcd17047c0460010004210200020c2
:020000040000fa
:1093540070b5050000f0dcfb002d14db6b090b4e2f
:109364009a0094591f222a40d44001210c40914074
:1093740020339b009951bff34f8fbff36f8f00f0e1
:10938400d0fb200070bd0024f9e7c04600e100e0f6
:020000040000fa
:10939400431e033311d84ff6ff730340042b0ed83a
:1093a40059010a4a5218d26990420ad10a0007495f
:1093b400525c42b15b01c81870470020fce70020f2
:1093c400fae70020f8e70020f6e7c0462020002056
:020000040000fa
:1093d40070b505000d4c63689b69984760616069ce
:1093e40000f03afb040000f04bf9200000f026fbeb
:1093f4002800fff7b9f900b970bd00f089fb04003b
:10940400fff75efc200000f08cfbf5e72021002034
:020000040000fa
:10941400002b11d1002a0fd1002900d1002802d03d
:109424000021c943081c07b4024802a14018029055
:1094340003bdc046ad07000003b4684601b50298f9
:10944400fef76afe019b9e4602b00cbc7047c04604
:020000040000fa
:10945400f7b5040007000026019148340cb9300028
:10946400febd6368a5680093009b013b009301d592
:109474002468f3e7ab89012b08d90e22ab5e0133d4
:1094840004d029003800019b984706436435ebe774
:020000040000fa
:1094940070b505000c00a8b100f0c2f800200a4a1b
:1094a40004210726a04208d0137e0b42fcd0138d62
:1094b4002b540130538b3342f4d0001b43425841a8
:0c94c400c0b270bd0020fce7000c0042ac
:020000040000fa
:1094d0001c2101231b04984201d3000c10391b0ae4
:1094e000984201d3000a08391b09984201d30009a8
:1094f000043902a2105c40187047c04604030202ff
:0c9500000101010100000000000000005b
:020000040000fa
:10950c0070b5050000f0d0f8012468b12800fff711
:10951c003bff040078b1437843b90023237563758e
:10952c002370002400f05ef8200070bdfff7eefd04
:0a953c0000236370f1e70124f4e757
:020000040000fa
:02954600fee73e
:020000040000fa
:109548000a4b0b4a1a600b4a9a81c02292025a604f
:109558001a00d369002bfcd1044a136802210b437b
:109568001360d369002bfcd17047c046000c004241
:089578000401104141f1ffff65
:020000040000fa
:10958000f8b51f008b8905000c001600db0505d51a
:109590000e23c95e0022022300f084f9a389054a44
:1095a00028001340a38132000e23e15e3b0000f04f
:0895b00055f9f8bdffefffffc4
:020000040000fa
:1095b80070b50c00002519b112b11500022801d9a7
:1095c800280070bd074b23b11100200000e000bf48
:1095d800f6e716002078013e00f057fa0134002e15
:0895e800f8d1ede700000000de
:020000040000fa
:1095f0000a4b1b7a5bb2002b07db5a091f210b4079
:10960000012199409300064a99502c23034ad35cc8
:1096100013b901213423d1547047c04620210020c2
:0496200000e100e085
:020000040000fa
:109624000a4b588b0723184000b97047074b802218
:109634001a7607225a831b7e5b07f6d5034b042157
:109644001a8d1a7e0a42fbd1efe7c046000c004295
:020000040000fa
:1096540030b570b179b105004118084a0124137e70
:109664002342fcd02b7813850135a942f7d1012080
:1096740030bd0020fce70120fae7c046000c0042a0
:020000040000fa
:109684000a4b1b6b73b168b1002105e09a68801a1c
:1096940099609b6933b128b19a688242f6d39a687b
:1096a400101a9860014b5a691a61704720210020f2
:020000040000fa
:1096b40010b52c23094ad35c012023b93423d35c8d
:1096c4000020012b00d010bd130000213422995436
:1096d40008201856fff73cfe0120f4e72021002063
:020000040000fa
:1096e40010b5fff72fff00f0a5f8fff711fe0549ad
:1096f4000020fff793fa044b186000f037fa00f0eb
:0c97040087f810bd949b0000002000209e
:020000040000fa
:10971000094a537980210b435371110004220b69cc
:109720001a42fcd104491f224b799343002bfbd1f1
:0c973000014b58697047c0460010004211
:020000040000fa
:10973c0010b5084b5b7a5bb1064b987ac0b23322fa
:10974c009a7228b1044b1b6813b1034a51689847ad
:0c975c0010bdc04600100042102000208c
:020000040000fa
:1097680070b564254a1e55430e0029007031fff775
:109778009bf9040040b100212a00016046600c30ca
:0c978800a060643200f0d4f9200070bd35
:020000040000fa
:1097940070b50c000e25495f00f082f8a389421cc5
:1097a40003d1054a1340a38170bd41f20002134363
:0c97b400a3816065f8e7c046ffefffffef
:020000040000fa
:1097c000074a13684bb107491818884202d810603d
:1097d0001800704701204042fbe7034b1360f2e79b
:0c97e00080210020882300208821002028
:020000040000fa
:1097ec0070b50c000e25495f00f068f8002803db0b
:1097fc00636d1b18636570bda389024a1340a38176
:08980c00f9e7c046ffefffff82
:020000040000fa
:10981400064b40f220301a5805491140c022120468
:109824000a431a5004225a607047c04600e100e01f
:04983400ffff00ff33
:020000040000fa
:10983800064a00231360936047f6ff4151600621f2
:109848001160034a936013607047c04610e000e05f
:0498580004200020c8
:020000040000fa
:10985c0070b50500080011000022054c22601a00aa
:10986c0000f0b2f9431c02d1236803b12b6070bd28
:04987c001c2000208c
:020000040000fa
:10988000002370b5064c050008001100236000f0ad
:1098900091f9431c02d1236803b12b6070bdc0460f
:0498a0001c20002068
:020000040000fa
:1098a40070b50500080011000022054c22601a0062
:1098b40000f086f9431c02d1236803b12b6070bd0c
:0498c4001c20002044
:020000040000fa
:1098c80070b50500080011000022054c22601a003e
:1098d80000f078f9431c02d1236803b12b6070bdf6
:0498e8001c20002020
:020000040000fa
:1098ec0070b5002661b15ab1160048b90c001500cc
:1098fc00012000f0bbf8013d20700134002df7d1a0
:04990c00300070bdfa
:020000040000fa
:109910000000000000000000000000000000000047
:109920000000000000000000000000000000000037
:020000040000fa
:109930000000000000000000000000000000000027
:109940000000000000000000000000000000000017
:020000040000fa
:109950000000000000000000000000000000000007
:1099600000000000000000000000000000000000f7
:020000040000fa
:10997000002370b5054c050008002360fff720ffa9
:10998000431c02d1236803b12b6070bd1c20002052
:020000040000fa
:10999000002370b5054c05000800236000f006f9af
:1099a000431c02d1236803b12b6070bd1c20002032
:020000040000fa
:1099b000002370b5054c05000800236000f0fef898
:1099c000431c02d1236803b12b6070bd1c20002012
:020000040000fa
:1099d000659b0000099a0000259a00009d9b0000ed
:0c99e000c59a0000d99a00001197000001
:020000040000fa
:1099ec0010b5054b9a6801329a601b6813b1024a94
:0c99fc005068984710bdc04604200020b1
:020000040000fa
:109a0800054a136802210b431360110002220b69f7
:0c9a18001a42fcd17047c046001000420a
:020000040000fa
:109a2400054a136802218b431360110002220b695b
:0c9a34001a42fcd17047c04600100042ee
:020000040000fa
:109a4000054a536ac0185062834200d87047936a2f
:0c9a500001339362fae7c0462021002099
:020000040000fa
:109a5c00054b1b69834203d3034b1b69c01a704728
:0c9a6c00014b1b69c01afae72021002002
:020000040000fa
:109a780000b583b000230193012101a8fff706fd7b
:0a9a88000028f9d0019803b000bdda
:020000040000fa
:109a920000b583b06b46d87101216b46d81dfff724
:0a9aa200d8fd0028f8d003b000bd85
:020000040000fa
:109aac0054696d65722062796c207679766f6c6181
:089abc006e203a2d290d000077
:020000040000fa
:109ac400034bd861190040220b691a42fcd170473c
:049ad400001000423c
:020000040000fa
:109ad800034b1862190080220b691a42fcd17047a7
:049ae8000010004228
:020000040000fa
:109aec00034b1b7813b90122014b1a707047c04607
:049afc00182000200e
:020000040000fa
:109b000010b5034b01001868fef708ff10bdc046f2
:049b1000742100209c
:020000040000fa
:109b1400eff3108072b6bff35f8f43425841c0b277
:029b2400704788
:020000040000fa
:109b260018b972b6bff35f8f7047bff35f8f62b627
:029b3600fae74c
:020000040000fa
:109b380003008218934200d1704719700133f9e786
:020000040000fa
:109b480010b50249fff782fc10bdc04675900000b1
:020000040000fa
:0c9b58000122014b1a707047862100208a
:020000040000fa
:0c9b6400014b1860596070471020002071
:020000040000fa
:0c9b70000022014b1a70704718200020e2
:020000040000fa
:0c9b7c0010b50e23c95efff705ff10bdf9
:020000040000fa
:0c9b880042f2000300204b607047c04612
:020000040000fa
:089b9400d0990000220000003e
:020000040000fa
:089b9c00004870470048e80191
:020000040000fa
:089ba40010b5fff7a1ff10bd91
:020000040000fa
:089bac0010b500f015f810bd22
:020000040000fa
:089bb40010b5fff7e7ff10bd3b
:020000040000fa
:089bbc0010b500f015f810bd12
:020000040000fa
:089bc40010b500f013f810bd0c
:020000040000fa
:089bcc0010b5fff78dfe10bd7e
:020000040000fa
:089bd40010b5fff7effc10bd16
:020000040000fa
:089bdc00012040427047c04621
:020000040000fa
:049be4007047c046c0
:020000040000fa
:049be800c020002079
:020000040000fa
:049bec00012070479d
:020000040000fa
:049bf000002070479a
:020000040000fa
:029bf4007047b8
:020000040000fa
:029bf6007047b6
:00000001FF
